:100000000C94D8000C94F5000C94F5000C94F500B9
:100010000C94F5000C94F5000C94F5000C94F5008C
:100020000C94F5000C940B040C94F5000C94F50062
:100030000C94F5000C94EA040C94F5000C94F50073
:100040000C94F5000C94F5000C94F5000C94F7005A
:100050000C94F500CC02EC03CF02EC03D202EC03CB
:10006000D402EC03EC03EC03EC03EC03EC03EC0331
:10007000D602EF02DB02EF02E502EF02EA02EF0234
:10008000EC03EC03EC03EC03EC03EC03EC03EC03F8
:10009000F202F702FC02010306030B03100315032F
:1000A000EC03EC03EC03EC03EC03EC03EC03EC03D8
:1000B0001A031F03240329032E03330338033D03CC
:1000C000420353035C03650368037D0386038F03C8
:1000D0009803A103AA03B303BC03C503D103DE0342
:1000E000BC03C503D103DE03EC03EC03EC03EC0318
:1000F000EC03EC03EC03EC03EC03EC03EC03EC0388
:10010000EC03EC03EC03EC03EC03EC03EC03EC0377
:10011000EC03EC03EC03EC03EC03EC03EC03EC0367
:10012000EC03EC03EC03EC03EC03EC03EC03EC0357
:10013000EC03EC03EC03EC03EC03EC03EC03EC0347
:10014000EC03EC03EC03EC03EC03EC03EC03EC0337
:10015000EC03EC03EC03EC03EC03EC03EC03EC0327
:10016000EC03EC03EC03EC03EC03EC03EC03EC0317
:10017000EC03EC03EC03EC03E70305A84CCDB2D48D
:100180004EB93836A9020C50B9918688083CA6AA07
:10019000AA2ABE000000803F4546476566670020EA
:1001A0002B2D2E3031323334353637383968000054
:1001B00011241FBECFE5D8E0DEBFCDBF10E0A0E622
:1001C000B0E0EEE5F5E202C005900D92A837B10768
:1001D000D9F721E0A8E7B0E001C01D92A636B2072A
:1001E000E1F70E94DF050C94AD120C9400001F9201
:1001F0000F920FB60F9211242F933F934F935F935B
:100200006F937F938F939F93AF93BF93EF93FF93DE
:1002100081B1887F803881F040F4803609F0E5C2F2
:1002200085EC86BF1092E600E5C2883A09F4A7C1C2
:10023000883B09F4A4C1D9C28091E600893209F44F
:100240003CC108F04BC0883009F4CFC0F0F48330D3
:1002500009F4F1C070F4813009F4EDC008F0A1C0D8
:1002600083B18093E6008091E60081508093E600A0
:10027000B1C2853009F4DFC008F49FC0863009F4AC
:10028000A8C0873009F4D7C0A8C2843209F4D3C00B
:10029000C8F4813209F4B5C020F4803209F4CBC02F
:1002A0009CC2823209F4C7C0833209F096C283B17E
:1002B0002091A60090E0922B9093CA008093C900F1
:1002C00081E0F3C0863209F4B6C008F4A7C08732D3
:1002D00009F4B5C0883209F4EBC07FC2833509F454
:1002E00003C1F8F48E3209F4E8C060F48B3209F4EB
:1002F000B3C008F4E2C08C3209F4DAC08D3209F4DC
:10030000DCC06BC2803509F4D3C020F48F3209F40D
:10031000A3C063C2813509F4D0C0823509F4CDC0D1
:100320005CC2803909F41BC168F5853509F400C148
:1003300008F4F9C0863509F4FBC0873509F04DC2D1
:1003400023B180919E0090919F00A091A000B09158
:10035000A100BA2FA92F982F8827822B80939E0067
:1003600090939F00A093A000B093A1008093EC0015
:100370009093ED00A093EE00B093EF0081E08093A6
:10038000F00028C2823909F4F2C008F4ECC08339C5
:1003900009F4F1C08F3F09F020C283B18093E500DA
:1003A0001CC283B12091A60090E0922B9093E400B0
:1003B0008093E3001092D4000DC283B12091A60077
:1003C00090E0922B9093E2008093E1001092D30092
:1003D00001C283B12091A60090E0922B9093E0009F
:1003E0008093DF001092D200F5C183B12091A60066
:1003F00090E0922B9093DE008093DD001092D1006C
:10040000E9C183B12091A60090E0922B9093CC009B
:100410008093CB0081E08093D400DCC183B1209134
:10042000A60090E0922B9093C8008093C70081E0D3
:100430008093D200CFC183B18093A600CBC183B19A
:100440002091A60090E0922B9093C6008093C50067
:1004500081E08093D100BEC123B18091A200909130
:10046000A300A091A400B091A5006627782F892F42
:100470009A2F622B6093A2007093A3008093A40034
:100480009093A5002AE931E043E555E40E945C0F12
:100490000E943C0E7093CC006093CB007093CA0016
:1004A0006093C90081E08093D4008093D30092C10F
:1004B00083B190E0A0E0B0E00EC023B18091A20033
:1004C0009091A300A091A400B091A500BA2FA92FEC
:1004D000982F8827822B8093A2009093A300A0934B
:1004E000A400B093A50076C123B18091A2009091A1
:1004F000A300A091A400B091A500BA2FA92F982F16
:100500008827822B8093A2009093A300A093A4003D
:10051000B093A5008093E8009093E900A093EA00CF
:10052000B093EB0057C183B190E0A0E0B0E00EC003
:1005300023B180919E0090919F00A091A000B09166
:10054000A100BA2FA92F982F8827822B80939E0075
:1005500090939F00A093A000B093A1003BC183B1F2
:100560008093D00037C183B18093CF0033C183B172
:100570008093CE002FC183B18093CD002BC1809199
:10058000E60090E0FC013297E339F10508F024C160
:10059000E65DFF4F0C9428108AB59BB51AC188B54B
:1005A00099B517C183B515C18CB713C18091DB0014
:1005B0009091DC0004C08091D9009091DA00909372
:1005C0009D0080939C0093B905C18091D7009091C4
:1005D000D800F5CF8091D5009091D600F0CF8091D2
:1005E0009C00F7C08091CB009091CC00ECCF809123
:1005F000CB009091CC00EDC08091C9009091CA00D1
:10060000E2CF8091C9009091CA00E3C08091C700F9
:100610009091C800D8CF8091C7009091C800D9C0F0
:100620008091C5009091C600CECF8091C500909179
:10063000C600CFC08091C1009091C200C4CF80910C
:10064000C1009091C200C5C08091BF009091C000D0
:10065000BACF8091BF009091C000BBC08091BD0017
:100660009091BE00B0CF8091BD009091BE00B1C00E
:100670008091BB009091BC00A6CF8091BB0090916F
:10068000BC00A7C08091AB009091AC00A091AD00E0
:10069000B091AE008093A2009093A300A093A40019
:1006A000B093A50025C08091A2009091A300A091D5
:1006B000A400B091A50071C08091A2009091A30008
:1006C000A091A400B091A50074C08091A20081C047
:1006D0008091A7009091A800A091A900B091AA00D4
:1006E00080939E0090939F00A093A000B093A100E0
:1006F0008B2F9927AA27BB276CC080919E009091D1
:100700009F00A091A000B091A10047C080919E00E1
:1007100090919F00A091A000B091A1004AC080914B
:10072000AF009091B000A091B100B091B20051C063
:100730008091B7009091B800A091B900B091BA0033
:10074000D7CF8091B7009091B800A091B900B09137
:10075000BA0023C08091B7009091B800A091B90071
:10076000B091BA0026C08091B7009091B800A091D6
:10077000B900B091BA002DC08091B3009091B4003F
:10078000A091B500B091B600B3CF8091B300909125
:10079000B400A091B500B091B600CD01AA27BB2747
:1007A00018C08091B3009091B400A091B500B091B1
:1007B000B600892F9A2FAB2FBB270BC08091B300B7
:1007C0009091B400A091B500B091B60002C08091A4
:1007D000E70083B985EC02C013B885E886BF809135
:1007E000E6008F5F8093E60005C086B78B7E86BFEC
:1007F00085EC86BFFF91EF91BF91AF919F918F9153
:100800007F916F915F914F913F912F910F900FBE0C
:100810000F901F9018951F920F920FB60F921124F0
:100820002F933F934F935F938F939F9399B390FD33
:1008300002C080E001C083E091FF02C091E08927FF
:1008400020919B00281B20FF1FC080939B0080915C
:10085000D000422F4270882349F08091DB009091B4
:10086000DC00242F30E02150310908C08091DB00EA
:100870009091DC0021E030E0241B3109820F931FAE
:100880009093DC008093DB0099B392959F7090FD6C
:1008900002C080E001C083E091FF02C091E089279F
:1008A00020919A00281B20FF1FC080939A008091FE
:1008B000CF002270882359F08091D9009091DA00FE
:1008C00041E050E0421B5109840F951F09C08091FF
:1008D000D9009091DA0030E021503109820F931F46
:1008E0009093DA008093D90099B39695969590FDF0
:1008F00002C080E001C083E091FF02C091E089273F
:1009000020919900281B20FF1FC08093990080919F
:10091000CE002270882359F08091D7009091D800A2
:1009200041E050E0421B5109840F951F09C080919E
:10093000D7009091D80030E021503109820F931FE9
:100940009093D8008093D70099B3929596959695F9
:10095000937090FD02C080E001C083E0927011F0BE
:1009600091E0892720919800281B20FF1FC08093C9
:1009700098008091CD00422F4270882349F08091E9
:10098000D5009091D600242F30E02150310908C0C5
:100990008091D5009091D60021E030E0241B3109F0
:1009A000820F931F9093D6008093D5008091C3004F
:1009B0009091C40001969093C4008093C3009F91CE
:1009C0008F915F914F913F912F910F900FBE0F909C
:1009D0001F9018951F920F920FB60F9211248F93AC
:1009E0009F93EF93FF935F9B16C0E091F300F0910C
:1009F000F4008CB1808381E0E835F80730F431965B
:100A0000F093F400E093F30006C085EF90E090933C
:100A1000F4008093F300FF91EF919F918F910F90DD
:100A20000FBE0F901F9018959C018AB188618AB9FA
:100A3000579A80B5866080BD40E050E084E0220F88
:100A4000331F441F551F8A95D1F760E072E18AE792
:100A500090E00E940910DA01C9010197A109B109CA
:100A6000892F9A2FAB2FBB27A7FDBA9580BD2150A8
:100A700029B985EF90E09093F2008093F100909374
:100A8000F4008093F30008955D9BFECFFC0180810C
:100A90008CB90895CF93DF931F92CDB7DEB78983CA
:100AA000CE0101960E94440580E090E00F90DF9116
:100AB000CF910895CF93DF93EC01CE012196FC01F5
:100AC0002081222319F00E944405F7CFDF91CF91B6
:100AD00008955F9BFECF8CB190E008950C9469055A
:100AE0006EE675E08AE495E00C945B10CF93DF939B
:100AF000FC01E253FF4FA081B181EC01C453DF4FF1
:100B000028813981A217B307A1F05D9B12C02C91F7
:100B10002CB920813181AC0145535F4F2417350733
:100B200018F42F5F3F4F03C09C0128593F4F31837A
:100B30002083E091F100F091F2002091F3003091D8
:100B4000F4002E173F07C1F1DC01AC59BF4FCD9126
:100B5000DC911197208128836D917C9111979C01E4
:100B60002B523F4FE9013881EB012881321307C036
:100B70009C012C523F4FE90148814F5F48839C0103
:100B80002D593F4F6217730728F4EB012196CD933F
:100B9000DC9302C08D939C93D1E0E835FD0730F4DF
:100BA0003196F093F200E093F10006C085EF90E0FB
:100BB0009093F2008093F100DF91CF910895CF934D
:100BC000DF9300D000D0CDB7DEB788E087BB8CEFD5
:100BD00084BB8CEB81BB1092E50080E895E20E941B
:100BE00014050E94700580E582B986B78B7E86BFAA
:100BF00085EC86BF81EF8FBD89E08EBD1BBC1ABC22
:100C000019BC18BC89E785BD13BC83BF1CBE8EE62A
:100C100090E00E94D81085B78F7885BF84E089BFA7
:100C200078942224239433243A940FEF10E0809197
:100C3000E6008F3F41F48091E500853A21F4F89475
:100C4000E0E0F8E109958091F000882309F465C09F
:100C50006091EC007091ED008091EE009091EF00BA
:100C6000C090E800D090E900E090EA00F090EB003E
:100C70002BED3FE049E450E40E945C0F25E236E0B2
:100C800041E85EE30E945C0F20E030E040E05FE37B
:100C90000E945C0FA70196010E94690D6B017C0107
:100CA0006091E8007091E9008091EA009091EB007A
:100CB0009B01AC010E94690DA70196010E94680D7D
:100CC0001092F0002AE931E043E555E40E945C0F00
:100CD0000E943C0E7093CC006093CB007093CA00CE
:100CE0006093C9002AE931E043E555E4C701B60144
:100CF0000E945C0F0E943C0E7093C8006093C70076
:100D00007093C6006093C500F1E0F093D400F093B7
:100D1000D300F093D200F093D1008091C300909162
:100D2000C4008833914008F47EC51092C40010922C
:100D3000C300F894A090DB00B090DC008091960096
:100D400090919700A81AB90AC090D900D090DA0003
:100D50008091940090919500C81AD90AE090D7002C
:100D6000F090D8008091920090919300E81AF90ACF
:100D70006090D5007090D600809190009091910085
:100D8000681A790AB501882777FD8095982F0E9407
:100D90006F0E2AE037ED43E25CE30E94D40D0E941F
:100DA0003C0E7093C2006093C100B601882777FDA6
:100DB0008095982F0E946F0E2AE037ED43E25CE3A6
:100DC0000E94D40D0E943C0E7093C0006093BF003F
:100DD000B701882777FD8095982F0E946F0E2AE033
:100DE00037ED43E25CE30E94D40D0E943C0E709309
:100DF000BE006093BD00B301882777FD8095982FD2
:100E00000E946F0E2AE037ED43E25CE30E94D40DAE
:100E10000E943C0E7093BC006093BB007894B501B7
:100E20006C0D7D1D882777FD8095982F0E946F0E91
:100E30002AE931E043ED55E40E94D40D4B015C01F9
:100E4000B701660D771D882777FD8095982F0E9442
:100E50006F0E2AE931E043ED55E40E94D40D2B01D9
:100E60003C01C090AF00D090B000E090B100F09095
:100E7000B200A50194010E94680D25E236E041E828
:100E80005EE30E94D40D9B01AC01C701B6010E9434
:100E9000690D6B017C012BED3FE049EC50E40E94B1
:100EA000580F2BED3FE049EC50E418162CF4C70125
:100EB000B6010E94680D0EC0C701B6010E94CD0D9B
:100EC00087FF0AC02BED3FE049EC50E4C701B601B3
:100ED0000E94690D6B017C01A3019201C501B4015F
:100EE0000E94690D20E030E040E05FE30E945C0F6B
:100EF0004B015C01C701B6010E94D10D2B013C01E1
:100F0000C701B6010E94BF0F69837A838B839C83DC
:100F1000F894C092AF00D092B000E092B100F0928D
:100F2000B200C090B700D090B800E090B900F09047
:100F3000BA00A5019401C301B2010E945C0F9B019C
:100F4000AC01C701B6010E94690D6093B7007093B0
:100F5000B8008093B9009093BA00C090B300D090CD
:100F6000B400E090B500F090B600A501940169814D
:100F70007A818B819C810E945C0F9B01AC01C7012F
:100F8000B6010E94690D6093B3007093B400809322
:100F9000B5009093B6007894C090C100D090C20084
:100FA0008091BF009091C000C80ED91ED7FE03C02B
:100FB0003FEFC31AD30AD594C794E090BD00F090D8
:100FC000BE008091BB009091BC00E80EF91EF7FEB8
:100FD00003C08FEFE81AF80AF594E794B6016E0D96
:100FE0007F1D882777FD8095982F0E946F0E2AE934
:100FF00031E043ED55E40E94D40D4B015C01B70193
:101000006C197D09882777FD8095982F0E946F0EB7
:101010002BEB3CE047E255E40E94D40DF89480921B
:10102000AB009092AC00A092AD00B092AE00609385
:10103000A7007093A8008093A9009093AA007894C9
:101040008091DB009091DC00909397008093960054
:101050008091D9009091DA0090939500809394004C
:101060008091D7009091D800909393008093920044
:101070008091D5009091D60090939100809390003C
:101080008091D400813009F0ACC08091CB00909168
:10109000CC00892B89F41092E4001092E3001092A6
:1010A0008F0010928E0010928A0010928B00109286
:1010B0008C0010928D0095C0E091CB00F091CC0097
:1010C0008091C1009091C200E81BF90BFA83E9837B
:1010D0002F01662457FC6094762CC0908A00D09033
:1010E0008B00E0908C00F0908D00C40CD51CE61CA9
:1010F000F71CC0928A00D0928B00E0928C00F09294
:101100008D008091E3009091E400BC01882777FD79
:101110008095982F0E946F0E4B015C01C301B201B4
:101120000E946F0E2CEB34E743E15CE30E945C0FFE
:101130002B013C01C701B6010E946F0E2BE631ED79
:1011400046E05AE30E945C0F9B01AC01C301B2016F
:101150000E94690D6B017C0180918E0090918F003F
:1011600029813A81281B390BB901882777FD8095A1
:10117000982F0E946F0E2CE234ED4AE15DE30E944D
:101180005C0F9B01AC01C701B6010E94690D9B0178
:10119000AC01C501B4010E94690D0E943C0E709320
:1011A000E4006093E30089819A8190938F0080939B
:1011B0008E008091E3009091E4008F3F910531F023
:1011C0002CF01093E4000093E3000BC08091E30047
:1011D0009091E40081309F4F24F43092E4002092FB
:1011E000E3008091D300813009F0ACC08091C90048
:1011F0009091CA00892B89F41092E2001092E100CC
:10120000109289001092880010928400109285003C
:10121000109286001092870095C02091C9003091ED
:10122000CA008091BF009091C000281B390B3A83FF
:1012300029832901662457FC6094762CC090840091
:10124000D0908500E0908600F0908700C40CD51CFB
:10125000E61CF71CC0928400D0928500E0928600C4
:10126000F09287008091E1009091E200BC01882714
:1012700077FD8095982F0E946F0E4B015C01C30192
:10128000B2010E946F0E2CEB34E743E15CE30E9455
:101290005C0F2B013C01C701B6010E946F0E2BE6CB
:1012A00031ED46E05AE30E945C0F9B01AC01C301A3
:1012B000B2010E94690D6B017C01809188009091C0
:1012C0008900E981FA81E81BF90BBF01882777FDC6
:1012D0008095982F0E946F0E2CE234ED4AE15DE379
:1012E0000E945C0F9B01AC01C701B6010E94690D11
:1012F0009B01AC01C501B4010E94690D0E943C0E26
:101300007093E2006093E10029813A813093890073
:10131000209388008091E1009091E2008F3F910539
:1013200031F02CF01093E2000093E1000BC08091AB
:10133000E1009091E20081309F4F24F43092E2006E
:101340002092E1008091D200813009F0B0C08091FC
:10135000C7009091C800892B89F41092E000109288
:10136000DF00109283001092820010927E00109293
:101370007F00109280001092810099C08091C70078
:101380009091C8009A8389838091BD009091BE009E
:10139000E981FA81E81BF90BFA83E9832F016624BE
:1013A00057FC6094762CC0907E00D0907F00E09037
:1013B0008000F0908100C40CD51CE61CF71CC09284
:1013C0007E00D0927F00E0928000F09281008091B8
:1013D000DF009091E000BC01882777FD8095982F71
:1013E0000E946F0E4B015C01C301B2010E946F0E9F
:1013F0002CEB34E743E15CE30E945C0F2B013C01E2
:10140000C701B6010E946F0E2BE631ED46E05AE3AC
:101410000E945C0F9B01AC01C301B2010E94690DE7
:101420006B017C01809182009091830029813A8137
:10143000281B390BB901882777FD8095982F0E94CA
:101440006F0E2CE234ED4AE15DE30E945C0F9B01DC
:10145000AC01C701B6010E94690D9B01AC01C50139
:10146000B4010E94690D0E943C0E7093E0006093ED
:10147000DF0089819A81909383008093820080911C
:10148000DF009091E0008F3F910531F02CF0109338
:10149000E0000093DF000BC08091DF009091E0003E
:1014A00081309F4F24F43092E0002092DF00809141
:1014B000D100813009F0ACC08091C5009091C60088
:1014C000892B89F41092DE001092DD0010927D00CD
:1014D00010927C00109278001092790010927A009D
:1014E00010927B0095C02091C5003091C60080917C
:1014F000BB009091BC00281B390B3A83298329013A
:10150000662457FC6094762CC0907800D0907900C7
:10151000E0907A00F0907B00C40CD51CE61CF71C10
:10152000C0927800D0927900E0927A00F0927B002D
:101530008091DD009091DE00BC01882777FD8095C9
:10154000982F0E946F0E4B015C01C301B2010E94F3
:101550006F0E2CEB34E743E15CE30E945C0F2B0140
:101560003C01C701B6010E946F0E2BE631ED46E04B
:101570005AE30E945C0F9B01AC01C301B2010E94BF
:10158000690D6B017C0180917C0090917D00E98167
:10159000FA81E81BF90BBF01882777FD8095982F0A
:1015A0000E946F0E2CE234ED4AE15DE30E945C0F75
:1015B0009B01AC01C701B6010E94690D9B01AC0102
:1015C000C501B4010E94690D0E943C0E7093DE00BB
:1015D0006093DD0029813A8130937D0020937C0067
:1015E0008091DD009091DE008F3F910531F02CF06D
:1015F0001093DE000093DD000BC08091DD00909120
:10160000DE0081309F4F24F43092DE002092DD0016
:101610008091E3009091E400209166003091670092
:1016200028173907B9F18091E3009091E400892BE4
:1016300019F485B38C6017C08091D000811107C068
:101640008091E3009091E4001816190654F08091FF
:10165000D000882351F08091E3009091E40097FF3F
:1016600004C085B3837F85BB02C0AA98AB9A8091E2
:10167000E3009091E400909367008093660080916E
:10168000E3009091E40097FF03C091958195910943
:101690009BBD8ABD8091E1009091E20020916400A1
:1016A0003091650028173907B9F18091E1009091D8
:1016B000E200892B19F485B3806317C08091CF00B5
:1016C000811107C08091E1009091E200181619067F
:1016D00054F08091CF00882351F08091E1009091E7
:1016E000E20097FF04C085B38F7C85BB02C0AC9835
:1016F000AD9A8091E1009091E20090936500809313
:1017000064008091E1009091E20097FF03C0919501
:101710008195910999BD88BD8091DF009091E0008D
:10172000209162003091630028173907B1F1809150
:10173000DF009091E000892B19F485B3806C17C00D
:101740008091CE00811107C08091DF009091E00070
:101750001816190654F08091CE00882351F080911C
:10176000DF009091E00097FF04C085B38F7385BBC5
:1017700002C0AE98AF9A8091DF009091E000909304
:101780006300809362008091DF009091E00097FFFA
:1017900003C091958195910983BD8091DD00909161
:1017A000DE00209160003091610028173907B1F107
:1017B0008091DD009091DE00892B19F482B38C605A
:1017C00017C08091CD00811107C08091DD009091FC
:1017D000DE001816190654F08091CD00882351F0D0
:1017E0008091DD009091DE0097FF04C082B3837F7B
:1017F00082BB02C09298939A8091DD009091DE00A6
:1018000090936100809360008091DD009091DE00F4
:1018100097FF03C09195819591098CBF8091E70056
:101820008F5F8093E70085B7806885BF889585B70F
:101830008F7785BFFCC96F927F929F92AF92BF92C4
:10184000CF92DF92EF92FF920F931F93CF93DF938C
:10185000CDB7DEB72C970FB6F894DEBF0FBECDBF65
:101860008C017B013A01FC0117821682838181FF82
:1018700019C1CE0101965C01F801D380F701D3FCB8
:101880002591D3FE21917F01222309F407C125323E
:1018900049F4D3FC2591D3FE21917F01253211F02B
:1018A000912C1BC0B801822F90E00E94A61063010A
:1018B0003601E2CF222309F4F1C0622F70E08FE9F4
:1018C00091E02C870E9450102C85892B49F0F7015C
:1018D000D3FC2591D3FE21917F0197FEEBCF0CC065
:1018E000233221F4F92DF0619F2EF1CF2C3639F4FB
:1018F000292D2068922EEBCF222309F4CFC0622F2E
:1019000070E088E991E02C870E9450102C85892B8B
:1019100041F06301F4E0CF0ED11CB8018FE390E0F9
:1019200012C0233641F0233789F0233521F5F92DF4
:10193000F1609F2E0BC0630122E0C20ED11CB801E2
:10194000F301808191810E94A610B2CF630122E051
:10195000C20ED11CF30160807180F30190FC85916F
:1019600090FE81913F01882309F4A2CFB80190E055
:101970000E94A610F2CF243611F0293639F5630102
:1019800097FE09C0F4E0CF0ED11CF3016081718194
:10199000828193810AC0F2E0CF0ED11CF3016081F5
:1019A0007181882777FD8095982FF92DFF7E9F2ED6
:1019B00097FF09C090958095709561957F4F8F4FE7
:1019C0009F4FF0649F2E2AE030E038C02037A1F00E
:1019D00040F42835D1F02F3609F060C028E030E01F
:1019E00019C0253719F0283751F058C0292D2F7EFE
:1019F000922E2AE030E00EC0892D8061982E992D1C
:101A00009462992E20E130E005C0E92DE4609E2E1D
:101A100020E132E0630197FE09C0F4E0CF0ED11C53
:101A2000F301608171818281938108C0F2E0CF0E61
:101A3000D11CF3016081718180E090E0A5010E94DA
:101A40000511782E7A1896FE05C0B8018DE290E057
:101A50000E94A61094FE16C0FE01E70DF11D8081C4
:101A6000803381F0B80180E390E00E94A61092FEDE
:101A700009C0292D2072822F90E0B801885A9F4F0B
:101A80000E94A6107A94F501E70DF11D8081B8013E
:101A900090E00E94A6107110F5CF0ACFF801868160
:101AA000978102C08FEF9FEF2C960FB6F894DEBFA0
:101AB0000FBECDBFDF91CF911F910F91FF90EF909F
:101AC000DF90CF90BF90AF909F907F906F900895E0
:101AD0005058BB27AA270ED0A0C169D130F06ED1D3
:101AE00020F031F49F3F11F41EF45EC10EF4E09536
:101AF000E7FB54C1E92FB3D180F3BA17620773072C
:101B00008407950718F071F49EF5CBC10EF4E095AB
:101B10000B2EBA2FA02D0B01B90190010C01CA01A7
:101B2000A0011124FF27591B99F0593F50F4503E52
:101B300068F11A16F040A22F232F342F4427585F44
:101B4000F3CF469537952795A795F0405395C9F75C
:101B50007EF41F16BA0B620B730B840BBAF0915014
:101B6000A1F0FF0FBB1F661F771F881FC2F70EC0B3
:101B7000BA0F621F731F841F48F487957795679586
:101B8000B795F7959E3F08F0B3CF9395880F08F06F
:101B90009927EE0F979587950895DCD008F481E09A
:101BA000089514D1E3954AC10CD037C107D140F054
:101BB000FED030F021F45F3F19F0F0C0511172C136
:101BC000F3C04DD198F39923C9F35523B1F3951B75
:101BD000550BBB27AA2762177307840738F09F5F4E
:101BE0005F4F220F331F441FAA1FA9F333D00E2EBD
:101BF0003AF0E0E830D091505040E695001CCAF72A
:101C000029D0FE2F27D0660F771F881FBB1F2617EE
:101C100037074807AB07B0E809F0BB0B802DBF01C1
:101C2000FF2793585F4F2AF09E3F510568F0B6C0DA
:101C300039C15F3FECF3983EDCF386957795679565
:101C4000B795F7959F5FC9F7880F911D9695879572
:101C500097F90895E1E0660F771F881FBB1F621791
:101C600073078407BA0720F0621B730B840BBA0B4F
:101C7000EE1F88F7E095089504D06894B11112C161
:101C80000895F5D088F09F5790F0B92F9927B75154
:101C9000A0F0D1F0660F771F881F991F1AF0BA9530
:101CA000C9F712C0B13081F0FCD0B1E00895F9C09D
:101CB000672F782F8827B85F39F0B93FCCF3869526
:101CC00077956795B395D9F73EF490958095709583
:101CD00061957F4F8F4F9F4F0895E89409C097FB00
:101CE0003EF490958095709561957F4F8F4F9F4FF3
:101CF0009923A9F0F92F96E9BB279395F695879537
:101D000077956795B795F111F8CFFAF4BB0F11F4F9
:101D100060FF1BC06F5F7F4F8F4F9F4F16C08823A0
:101D200011F096E911C0772321F09EE8872F762FD6
:101D300005C0662371F096E8862F70E060E02AF017
:101D40009A95660F771F881FDAF7880F9695879503
:101D500097F90895990F0008550FAA0BE0E8FEEFD8
:101D600016161706E807F907C0F012161306E4075F
:101D7000F50798F0621B730B840B950B39F40A2658
:101D800061F0232B242B252B21F408950A2609F436
:101D9000A140A6958FEF811D811D089597F99F673A
:101DA00080E870E060E008959FEF80EC08950024E3
:101DB0000A941616170618060906089500240A94B0
:101DC00012161306140605060895EECF50D0E8F358
:101DD000E894E0E0BB279F57F0F02AED3FE049ECA4
:101DE00006C0EE0FBB0F661F771F881F28F0B23AA0
:101DF00062077307840728F0B25A620B730B840BD7
:101E0000E3959A9572F7803830F49A95BB0F661F68
:101E1000771F881FD2F79048BAC0092E0394000C90
:101E200011F4882352F0BB0F40F4BF2B11F460FF74
:101E300004C06F5F7F4F8F4F9F4F0895EF93E0FF78
:101E400006C0A2EA2AED3FE049EC5FEB53DEE5DF96
:101E50000F90039401FC9058EAE7F1E0A4C057FD0D
:101E60009058440F551F59F05F3F71F04795880F08
:101E700097FB991F61F09F3F79F08795089512169F
:101E800013061406551FF2CF4695F1DF08C016164B
:101E900017061806991FF1CF8695710561050894FC
:101EA0000895E894BB2766277727CB0197F9089513
:101EB00051DF08F48FEF08950BD0AFCF78DF28F013
:101EC0007DDF18F0952309F069CF6ECF1124EACF9A
:101ED000C6DFA0F3959FD1F3950F50E0551F629F89
:101EE000F001729FBB27F00DB11D639FAA27F00D73
:101EF000B11DAA1F649F6627B00DA11D661F829F9A
:101F00002227B00DA11D621F739FB00DA11D621F7E
:101F1000839FA00D611D221F749F3327A00D611D9B
:101F2000231F849F600D211D822F762F6A2F11247D
:101F30009F5750408AF0E1F088234AF0EE0FFF1FD0
:101F4000BB1F661F771F881F91505040A9F79E3F07
:101F5000510570F023CFA6CF5F3FECF3983EDCF342
:101F6000869577956795B795F795E7959F5FC1F744
:101F7000FE2B880F911D9695879597F908959F934D
:101F800025DF0F9007FCEE5F59CF9F3F31F0915056
:101F900020F4879577956795B795880F911D96954D
:101FA000879597F908959F938F937F936F93FF93EE
:101FB000EF939B01AC0180DFEF91FF9105D02F9152
:101FC0003F914F915F9178CFDF93CF931F930F9302
:101FD000FF92EF92DF927B018C01689405C0DA2EAC
:101FE000EF0176DFFE01E894A591259135914591A9
:101FF0005591AEF3EF017EDDFE019701A801DA9461
:1020000079F7DF90EF90FF900F911F91CF91DF91C3
:102010000895052E97FB1EF400940E94201057FD92
:1020200007D00E942E1007FC03D04EF40C94201011
:1020300050954095309521953F4F4F4F5F4F0895F4
:1020400090958095709561957F4F8F4F9F4F089524
:10205000EE0FFF1F0590F491E02D0994A1E21A2ED6
:10206000AA1BBB1BFD010DC0AA1FBB1FEE1FFF1F3C
:10207000A217B307E407F50720F0A21BB30BE40B8C
:10208000F50B661F771F881F991F1A9469F76095D3
:102090007095809590959B01AC01BD01CF0108958D
:1020A000FC010590061621F00020D9F7C001089523
:1020B0003197CF0108950F931F93CF93DF93EC01D6
:1020C0008B01009731F46115710519F480E090E0FF
:1020D00038C06EE070E081E090E00E946311FC0186
:1020E0000097A1F380E883830115110571F0138730
:1020F000028781E8838380915C0190915D01892B47
:1021000021F4F0935D01E0935C012097C9F0D18741
:10211000C08783818260838380915E0190915F019B
:10212000892B71F4F0935F01E0935E01809160016F
:1021300090916101892B21F4F0936101E09360019A
:10214000CF01DF91CF911F910F9108950F931F93AE
:10215000CF93DF93182F092FEB018B8181FD03C0F3
:102160008FEF9FEF20C082FF10C04E815F812C81D6
:102170003D81421753077CF4E881F9819F012F5F6D
:102180003F4F39832883108306C0E885F985812F66
:102190000995892B29F72E813F812F5F3F4F3F8380
:1021A0002E83812F902FDF91CF911F910F91089552
:1021B0000F931F93CF93DF93E0915E01F0915F0146
:1021C000238121FF1BC0EC0100E010E089916091A8
:1021D0005E0170915F01DB011896ED91FC911997FA
:1021E000882331F00995892B89F30FEF1FEFEECF8C
:1021F0008AE00995892B11F4C80102C08FEF9FEF87
:10220000DF91CF911F910F910895FA01AA272830ED
:1022100051F1203181F1E8946F936E7F6E5F7F4FB3
:102220008F4F9F4FAF4FB1E03ED0B4E03CD0670F2F
:10223000781F891F9A1FA11D680F791F8A1F911D82
:10224000A11D6A0F711D811D911DA11D20D009F4D2
:1022500068943F912AE0269F11243019305D319314
:10226000DEF6CF010895462F4770405D4193B3E0FD
:102270000FD0C9F7F6CF462F4F70405D4A3318F0A4
:10228000495D31FD4052419302D0A9F7EACFB4E055
:10229000A6959795879577956795BA95C9F700970D
:1022A0006105710508959B01AC010A2E06945795AE
:1022B000479537952795BA95C9F7620F731F841F05
:1022C000951FA01D08950F931F93CF93DF93869FB3
:1022D0008001879F100D969F100D1124C8010E9448
:1022E0007F11EC01009729F0A80160E070E00E94E6
:1022F000A612CE01DF91CF911F910F910895CF9338
:10230000DF938230910510F482E090E0E091640167
:10231000F091650120E030E0A0E0B0E0309739F1C5
:102320004081518148175907B8F04817590771F48F
:1023300082819381109729F013969C938E93129724
:102340002CC0909365018093640127C0211531054D
:1023500031F04217530718F0A901DB0101C0EF016A
:102360009A01BD01DF010280F381E02DD7CF211555
:102370003105F9F0281B390B2430310580F48A81AE
:102380009B816115710521F0FB019383828304C059
:102390009093650180936401FE01329644C0FE0172
:1023A000E20FF31F819391932250310939832883DF
:1023B0003AC02091620130916301232B41F42091B6
:1023C0006A0030916B003093630120936201209189
:1023D0006800309169002115310541F42DB73EB7F1
:1023E00040916C0050916D00241B350BE09162010F
:1023F000F0916301E217F307A0F42E1B3F0B28179F
:10240000390778F0AC014E5F5F4F2417350748F06D
:102410004E0F5F1F5093630140936201819391932C
:1024200002C0E0E0F0E0CF01DF91CF910895CF93BB
:10243000DF93009709F487C0FC0132971382128260
:10244000C0916401D0916501209781F42081318190
:10245000280F391F809162019091630182179307C1
:1024600079F5F0936301E09362016DC0DE0120E035
:1024700030E0AE17BF0750F412964D915C91139760
:102480009D014115510509F1DA01F3CFB383A28310
:1024900040815181840F951F8A179B0771F48D919C
:1024A0009C911197840F951F0296918380831296B9
:1024B0008D919C911397938382832115310529F483
:1024C000F0936501E09364013EC0D9011396FC933B
:1024D000EE9312974D915D91A40FB51FEA17FB077C
:1024E00079F480819181840F951F0296D90111960C
:1024F0009C938E938281938113969C938E931297D3
:10250000E0E0F0E08A819B81009719F0FE01EC0188
:10251000F9CFCE01029628813981820F931F209135
:102520006201309163012817390769F4309729F463
:10253000109265011092640102C013821282D0933E
:102540006301C0936201DF91CF910895DC0101C066
:0E2550006D9341505040E0F70895F894FFCF8E
:10255E0000800080008000800000660120000D0ACF
:08256E0053746172740D00004A
:00000001FF
